:1000000001308A009B290000D3346D38EC32202A5D
:10001000E832F236EF36653AE8327210A0060A008E
:10002000D63C73366532EE3220265321A0126C2C5A
:10003000A0060A00A01320088316870083128713E6
:100040000830F80023280000F8173428F813B00C03
:1000500003188717031C8713781734287813F80BB5
:1000600027283228000087173F308400840B362869
:100070000000F81B2628781B2E280800831603177B
:100080008C170C140000000083120C087F39031930
:1000900082280313AC0003170D080313AD000317E8
:1000A0000F080313AE002C08B0001A202D08031708
:1000B0008D0003132E0803178F0083168C170C1462
:1000C0000000000083120C0D0E0D7F3903198228E9
:1000D0000313AC0003170D080313AD0003170F083B
:1000E0000313AE002C08B0001A202D0803178D0052
:1000F00003132E0803178F008D0A03198F0A0313A9
:100100003E28031703138A110A12072A0830F80041
:1001100000008711A01120088316870000008312B9
:10012000AC0D0712031C9A2820162008831687009E
:100130009E28831220122008831687000000831255
:10014000A0152008831687008312871DA528F80BA9
:10015000882800008711A01120088316870000005E
:1001600083122016200883168700000000008312E7
:10017000A0152008831687008312871DBD28F8016B
:100180000000071A78148711A01120088316870031
:10019000831207122012200883168700831208009A
:1001A0002C308400831300080319E3280230F80080
:1001B000F701F70BD928F80BD8289730F700F70B81
:1001C000DF28800BD62808000830AD007708AE0085
:1001D000201620088316870000008312A01520082F
:1001E000831687008312871DF328071A0314071E3E
:1001F0000310F80D0000A011200883168700831259
:100200008711AD0BE8282016200883168700000010
:10021000831207122E0803191229201220088316B0
:10022000870083120000A015200883168700831220
:10023000871D182900008711A01120088316870048
:1002400000008312071220122008831687008312F1
:100250000800AD1B3B290F30F7002C0EF7050A30C4
:100260007702031836293030F70738292D08F707A9
:100270007708B0001A200F30AC050A302C020318A2
:10028000432930304529AD132D08AC072C08B000A8
:100290001A200800831603178C170C1400000000A6
:1002A0000318792983120C087F390313AD00031753
:1002B0000D080313AE0003170F080313AF002D083A
:1002C000B0001A202E0803178D0003132F08031700
:1002D0008F0083168C170C14000000008312031388
:1002E000AC0B73297629831603177929982983166D
:1002F000031783120C0D0E0D7F390313AD00031786
:100300000D080313AE0003170F080313AF002D08E9
:10031000B0001A202E0803178D0003132F080317AF
:100320008F008D0A03198F0A03100313AC0B4A299F
:100330008A110A12022C840183131F308305713045
:1003400083168F000F088312A013200883168700DE
:1003500083128717831603170908C039890003130E
:100360001F129F1200300317880083128701880133
:100370008901FF300313A000831603170908C03951
:10038000890003131F129F12003003178800831285
:1003900003131F139F1383169F1383121F149412AA
:1003A000A0122008831687008312201620088316C7
:1003B00087008312A0112008831687000130831262
:1003C00094000030831694000108C7390838810072
:1003D000831290010030F8009200003083169200E2
:1003E0008312201520088316870083129701831635
:1003F0009B019C0101309D00831203178701880136
:10040000890104308D0000308F0003133E28A701BE
:10041000A901201620088316870000008312A0156A
:10042000200883168700000083120712201220087C
:1004300083168700000083128711A01120088316FD
:100440008700AA308312AC0086206130AC00862081
:10045000201620088316870000008312A0152008AC
:100460008316870000008312871D342A071220128A
:10047000200883168700000083128711A01120082E
:1004800083168700AA308312AC008620AC01862038
:10049000201220088316870000008312A015200870
:1004A000831687008312871D532A0000572A0000F5
:1004B0002016200883168700000001308312AC004C
:1004C000D020201620088316870000008312A01574
:1004D00020088316870000008312071220122008CC
:1004E00083168700000083128711A011200883164D
:1004F0008700AA308312AC0086203E30AC008620F4
:10050000201620088316870000008312A0152008FB
:100510008316870000008312871D8C2A0712201281
:10052000200883168700000083128711A01120087D
:1005300083168700AA308312AC0086205030AC00AE
:100540008620201220088316870000008312A01541
:100550002008831687008312871DAC2A0000B02A6A
:100560000000201620088316870000000130831247
:10057000AC00D020201620088316870000008312CC
:10058000A01520088316870000008312071220128E
:10059000200883168700000083128711A01120080D
:1005A00083168700AA308312AC0086203F30AC004F
:1005B0008620201620088316870000008312A015CD
:1005C00020088316870000008312871DE52A071282
:1005D0002012200883168700000083128711A011C3
:1005E000200883168700AA308312AC0086200230D0
:1005F000AC0086202012200883168700000083129A
:10060000A0152008831687008312871D052B000084
:10061000092B0000201620088316870000000130F7
:100620008312AC00D020201620088316870000001B
:100630008312A0152008831687000000831207127A
:100640002012200883168700000083128711A01152
:10065000200883168700AA308312AC00862043301E
:10066000AC00862020162008831687000000831225
:10067000A01520088316870000008312871D3E2BDB
:1006800007122012200883168700000083128711AA
:10069000A011200883168700AB308312AC0086209F
:1006A000F701E4207808AA002012200883168700AA
:1006B00000008312A0152008831687008312871D6F
:1006C0005F2B0000632B0000201620088316870094
:1006D0000000831220162008831687000000831272
:1006E000A01520088316870000008312071220122D
:1006F000200883168700000083128711A0112008AC
:1007000083168700AA308312AC0086204430AC00E8
:100710008620201620088316870000008312A0156B
:1007200020088316870000008312871D952B07126F
:100730002012200883168700000083128711A01161
:10074000200883168700AB308312AC008620F701A7
:10075000E4207808AB0020122008831687000000F0
:100760008312A0152008831687008312871DB62BDD
:100770000000BA2B00002016200883168700000016
:1007800001308312AC00D0205630B0001A204C301B
:10079000B0001A202030B0001A202B08AC003730EF
:1007A000AD0029212030B0001A200D30B0001A20F1
:1007B0000A30B0001A204C30B0001A204830B00087
:1007C0001A202030B0001A202A08AC003730AD00C3
:1007D00029212030B0001A200D30B0001A200A3034
:1007E000B0001A202A080A3C031D122C0130A7026F
:1007F000103003178D0000308F0003100D300313ED
:10080000AC004A292708AC003730AD002921203040
:10081000B0001A200D30B0001A200A30B0001A20A3
:10082000102CBE2C2016200883168700000083128F
:10083000A0152008831687000000831207122012DB
:10084000200883168700000083128711A01120085A
:1008500083168700AA308312AC0086204330AC0098
:100860008620201620088316870000008312A0151A
:1008700020088316870000008312871D3D2C071275
:100880002012200883168700000083128711A01110
:10089000200883168700AA308312AC0086200A3015
:1008A000AC008620201220088316870000008312E7
:1008B000A0152008831687008312871D5D2C000079
:1008C000612C000020162008831687000000831288
:1008D000201620088316870000008312A015200828
:1008E0008316870000008312071220122008831647
:1008F0008700000083128711A0112008831687004B
:10090000AA308312AC0086204430AC00862020162A
:1009100020088316870000008312A0152008831684
:10092000870000008312871D932C071220122008D5
:1009300083168700000083128711A01120088316F8
:100940008700AA308312AC0086205A30AC00862083
:10095000201220088316870000008312A0152008AB
:10096000831687008312871DB32C0000B72C00006C
:100970002016200883168700000083122016200806
:100980008316870000008312A015200883168700B5
:10099000000083120712201220088316870000002F
:1009A00083128711A011200883168700AA308312B2
:1009B000AC0086206030AC0086202016200883160C
:1009C000870000008312A01520088316870000000E
:1009D0008312871DE92C0712201220088316870036
:1009E000000083128711A011200883168700AA3007
:1009F0008312AC0086202708AC0086202012200835
:100A00008316870000008312A01520088316870034
:100A10008312871D092D00000D2D000020162008CF
:100A200083168700000001308312A7076430AC00F2
:060A3000D020092A63003A
:04400E00F52CFF3F4F
:00000001FF
